S01B00006F70656E626C745F656B5F6C6D3373383936322E737265632F
S113000048080020A12400007D2200007D22000079
S11300107D2200007D2200007D2200007D22000060
S11300207D2200007D2200007D2200007D22000050
S11300307D2200007D2200007D2200007D22000040
S11300407D2200007D2200007D2200007D22000030
S11300507D2200007D2200007D2200007D22000020
S11300607D2200007D2200007D2200007D22000010
S11300707D2200007D2200007D2200007D22000000
S11300807D2200007D2200007D2200007D220000F0
S11300907D2200007D2200007D2200007D220000E0
S11300A07D2200007D2200007D2200007D220000D0
S11300B07D2200007D2200007D2200007D220000C0
S11300C07D2200007D2200007D2200007D220000B0
S11300D07D2200007D2200007D2200007D220000A0
S11300E07D2200007D2200007D2200007D22000090
S11300F0DFF8B816884207D0DFF8B416884203D078
S1130100DFF8B016884201D1012070470020704703
S1130110DFF89816884208D0DFF89416884206D093
S1130120DFF89016884204D005E037207047382065
S11301307047392070474FF0FF30704770B582B078
S11301400546280B0003FFF7E3FF044614F1010FF3
S113015004D1F9210FF2686000F062FBDFF8580661
S1130160006801212246303A914011EA000602D08B
S1130170204600F097FB28680020009002E00098D9
S1130180401C009000980528F9DB2D68002E02D051
S1130190204600F049FB284676BD81B0016000206E
S11301A0009002E00098401C009000980528F9DBBC
S11301B001B07047F8B504460D46164600270BE01B
S11301C0E15D7F1CB74203DAE05D41EA00217F1C58
S11301D02846FFF7E2FF2D1DB742F1DBF1BDF8B56C
S11301E004460D46164600270AE02846FFF7A6FFF8
S11301F02D1DE0557F1CB74202DA000AE0557F1C32
S1130200B742F2DBF1BDF8B50446FFF771FF0028F1
S113021005D140F2D9110FF2A85000F001FB0121E1
S11302202046FFF7BAFF04F120052846FFF786FFB2
S11302300004FAD404F12406B0213046FFF7ADFFE0
S1130240002104F13400FFF7A8FF002104F1380075
S1130250FFF7A3FF012709E02846FFF76FFF00041B
S1130260FAD439462846FFF798FF7F1C212FF3DB89
S11302700C213046FFF791FF012609E02846FFF7DD
S11302805DFF0004FAD431462846FFF786FF761C4A
S1130290212EF3DB201DBDE8F2404FE710B50446E4
S11302A0FFF726FF002805D140F23A210FF2105043
S11302B000F0B6FA2046FFF741FF41084900204606
S11302C0BDE8104069E770B504460D460FF2F046EC
S11302D0FFF70EFF002804D14FF45971304600F0A7
S11302E09FFA002D04D140F26531304600F098FAAF
S11302F02868801E0F2804D340F26B31304600F08A
S11303008FFA6868002801D0092804D34FF45C717F
S1130310304600F085FAA868002801D0052804D3E7
S113032040F27531304600F07BFAE868B0F5806F32
S113033001D8002804D140F27B31304600F070FA35
S11303402046FFF7FBFE064646F041012046FFF734
S113035024FF6868401E000300F4E0402968491E39
S1130360090201F470610843A968491E890101F07A
S1130370C0010843E968491E01F03F01014304F14B
S11303800C00FFF70AFFE868401E800900F00F0127
S113039004F11800FFF701FF26F04001C80701D55A
S11303A0490849002046BDE87040F6E638B50446E1
S11303B00D46FFF79DFE002805D140F292510FF241
S11303C0004000F02DFA032D32D8DFE805F0020DCD
S11303D01925241D2046FFF7B1FE05466FF01F01C5
S11303E02046FFF7DAFE24E004F58070FFF7A6FE4E
S11303F0054604F58270FFF7A1FE45EA004518E0C2
S113040004F59070FFF79AFE054604F59270FFF725
S113041095FE45EA00450CE004F5B070FFF78EFE4A
S1130420054604F5B270FFF789FE45EA004500E091
S11304300025284632BD00002DE9FB4F0446154631
S11304400026FFF755FE002805D140F25F610FF248
S1130450703000F0E5F90198212801D2002805D177
S11304604FF4CC610FF2583000F0DAF99DF808002F
S113047000280DD001280BD0022809D0032807D06A
S1130480042805D040F266610FF2343000F0C8F958
S113049004F12000FFF752FE0004F9D42868B0F5F7
S11304A0006F04D2A968890801F0010100E001216C
S11304B04FF0930B3246009217469246904691466F
S11304C09DF80820042A00F29A80DFE802F0031560
S11304D0081823004FF4807A4FF400570126AB68C4
S11304E01A0722D56A688C46BCF1000F18D09046D2
S11304F0120CC2F30C0918E04FF4807AEFE74FF4C2
S113050000574FF4805A4FF6FF7841F6FF794FF0C9
S1130510D30BE4E74FF400574FF4905A0126DEE77B
S11305204FF000089200C2F30C0903F02802282AB5
S113053001D149F4004903F01802182A01D149F401
S1130540804913F0380F03D04AF4805A4BF0400B23
S11305504BF0200B002909D0014689B20091000C10
S1130560C0F30C0040F44040074305E08000C0F3B2
S11305700C0040F400400743EA6802F00F0040EA30
S11305800A0A980501D44AF0800AD80701D54AF42A
S1130590006A980701D54AF4806A002E04D004F159
S11305A03C012869FFF706FE594604F12400FFF7D1
S11305B0F4FD1FFA88F8414604F12800FFF7EDFD29
S11305C0494604F12C00FFF7E8FD6846018804F170
S11305D03000FFF7E2FD394604F13400FFF7DDFD9A
S11305E0514604F13800FFF7D8FD019800F03F01AF
S11305F004F1200003B0BDE8F04FFFF7CEBDBDE825
S1130600F78F2DE9F84F04460F4615461E46FFF7AF
S11306106FFD002805D140F2C1710FF2A41000F063
S1130620FFF8212F01D2002F05D140F2C2710FF241
S1130630901000F0F5F87321002E00D07B2104F116
S11306408400FFF7AAFD04F1800607F03F0739464E
S11306503046FFF7A2FD3046FFF770FD0004FAD4E0
S113066004F18800FFF76AFD804604F18C00FFF76F
S113067065FD81461FFA89F904F19000FFF75EFDDC
S1130680824604F19400FFF759FD83461FFA8BFB61
S113069004F19800FFF752FD80B20021A960C10562
S11306A002D45FEA8B4104D4C10504D55FEA8B41CF
S11306B001D44021A9605FEA4B410CD53F4901EACE
S11306C00B411FFA8AFA4AEA01012960A96841F03C
S11306D00401A96004E04FEAAB01C1F30A012960F7
S11306E0410403D5A96841F48071A960C1042DD5E2
S11306F05FEA4B410CD5314901EA09411FFA88F8F8
S113070048EA010169606FF0604291420CD108E04F
S11307104FEAA901C1F30A01696040F2FF729142F4
S113072002D1297A490603D4A96841F00801A960D5
S11307305FEA094103D5A96841F02801A9605FEA8D
S1130740494103D5A96841F01801A960010503D501
S1130750A96841F00101A960410503D5A96841F0E8
S11307600201A96001041DD500F00F02EA60287A95
S1130770400604D404F19C012869FFF730FD0421EC
S113078004F18400FFF709FD39463046FFF705FD03
S11307903046FFF7D3FC0004FAD4A86840F0800088
S11307A0A86001E00020E860BDE8F18F000004408B
S11307B0001004400020044004E100E00000FF1F9A
S11307C0433A5C576F726B5C736F667477617265E2
S11307D05C4F70656E424C545C5461726765745C26
S11307E044656D6F5C41524D434D335F4C4D335303
S11307F05F454B5F4C4D3353383936325F49415274
S11308005C426F6F745C6C69625C64726976657279
S11308106C69625C63616E6C69622E630000000047
S113082080B500F0B6F8FCE710B50446472C05D3B4
S11308304FF4D5710FF2F800FFF7F2FF042C05D145
S11308403748016841F48031016010BD052C05D1A1
S11308503348016841F40031016010BD062C05D114
S11308602F48016841F48021016010BD0F2C05D18F
S11308702C48016841F00201016010BDA4F1100090
S1130880202806D20120A4F11001884026490860DE
S113089010BD302C05D30120A4F130018840224939
S11308A0486010BD10B50446472C05D34FF4F771CA
S11308B00FF27C00FFF7B4FF042C05D1184801683F
S11308C021F48031016010BD052C05D11448016864
S11308D021F40031016010BD062C05D110480168D7
S11308E021F48021016010BD0F2C05D10D48016851
S11308F021F00201016010BDA4F11000202806D2ED
S11309000120A4F1100188400849086010BD302C72
S113091005D30120A4F1300188400449486010BD8A
S113092024ED00E010E000E000E100E080E100E000
S1130930433A5C576F726B5C736F66747761726570
S11309405C4F70656E424C545C5461726765745CB4
S113095044656D6F5C41524D434D335F4C4D335391
S11309605F454B5F4C4D3353383936325F49415202
S11309705C426F6F745C6C69625C64726976657208
S11309806C69625C696E746572727570742E630052
S113099070477047DFF85814884200F0A980DFF8E8
S11309A05414884200F0A480DFF84C14884200F00C
S11309B09F80DFF84814884200F09A80DFF84014E2
S11309C0884200F09580DFF83C14884200F0908063
S11309D0DFF83414884200F08B80DFF8301488424A
S11309E000F08680DFF82814884200F08180DFF868
S11309F0241488427CD0DFF82014884278D0DFF8B1
S1130A001C14884274D0DFF81814884270D0DFF8C0
S1130A10141488426CD0DFF81014884268D0DFF8D0
S1130A200C14884264D0DFF80814884260D0DFF8E0
S1130A30041488425CD0DFF80014884258D040285F
S1130A4056D0B0F1102F53D0DFF8F01388424FD0B6
S1130A50DFF8EC1388424BD0DFF8E813884247D024
S1130A60DFF8E413884243D0DFF8E01388423FD034
S1130A70B0F1101F3CD0DFF8D813884238D0DFF82B
S1130A80D413884234D0DFF8D013884230D0DFF852
S1130A90CC1388422CD0DFF8C813884228D0DFF862
S1130AA0C413884224D0DFF8C013884220D0DFF872
S1130AB0BC1388421CD0DFF8B813884218D0DFF882
S1130AC0B413884214D0DFF8B013884210D0DFF892
S1130AD0AC1388420CD0B0F1202F09D0DFF8A0135A
S1130AE0884205D0082803D0DFF89813884201D142
S1130AF0012070470020704710B50446FFF74AFFF5
S1130B00002805D14FF4FC710FF2C030FFF788FEC6
S1130B100FF21840210F50F821000168A2B2230CF3
S1130B2003F01F039A401143016010BD0138FDD149
S1130B3070477047F8B50446DFF84C53286810F046
S1130B40E04F06D02868DFF844130840B0F1805F16
S1130B5001D1002C7CD4286E296F20F4800040F44D
S1130B60006641F400672E662F67B00701D5A00721
S1130B7007D506F0010004F0010181F001010842EB
S1130B801AD064F0030006402E66002F05D507F046
S1130B907000302807D0702805D0002F08D406F044
S1130BA03000302804D14FF48050FFF7BFFF03E03A
S1130BB04FF40020FFF7BAFFDFF8D402304043F2CD
S1130BC0F071214041EA0006DFF8C8023840DFF83E
S1130BD0C81221400843E10001F0400141EA000746
S1130BE04020A865002F02D52F672E6601E02E66EF
S1130BF02F671020FFF79AFFDFF8A0023040DFF8DC
S1130C00A01221400843E10D61F3DC57610008D5CF
S1130C1040F4800027F48001DFF888222240114349
S1130C2001E027F0804122050CD44FF4004200E09B
S1130C30521E002A02D02B6D5B06F9D520F4006009
S1130C4021F40061286629671020BDE8F2406DE7B1
S1130C50F1BD70B4DFF830120A6E0B6F002B02D5B1
S1130C6003F0700001E002F0300000280AD01028E0
S1130C7031D0202856D030287BD060287CD07028F2
S1130C807DD07FE00FF2B020C2F3841450F824002A
S1130C90DFF8144204EA0305B5F1004F05D0002B38
S1130CA000F18380150500F180804D6E0E6816F00A
S1130CB0E04F06D00968DFF8D4613140B1F1805FBC
S1130CC062D1C5F34811891C484305F01F01891CF2
S1130CD0B0FBF1F061E0086810F0E04F06D0DFF8F7
S1130CE0AC010C680440B4F1805F02D1DFF8BC01B0
S1130CF0CEE70C680440DFF8B851AC4203D10C686D
S1130D00A4B2022C08D00C682040DFF8A841A0420D
S1130D1005D10868000402D1DFF89C01B8E7DFF8C8
S1130D209C01B5E7086810F0E04F06D0DFF85C01DD
S1130D300C680440B4F1805F02D1DFF88401A7E7B6
S1130D400C680440DFF86851AC4203D10C68A4B2CB
S1130D50022C08D00C682040DFF85841A04205D18D
S1130D600868000402D1DFF85C0191E7DFF858015C
S1130D708EE747F230508BE74FF4800088E74FF45A
S1130D80004085E7002031E0C5F34811484305F0F1
S1130D901F01491C4900B0FBF1F0690400D540086B
S1130DA0290400D5800842F4800251021ED5002B8C
S1130DB017D559000FD504EA0301B1F1004F03D050
S1130DC0002B08D4110506D44000C3F38651491CF6
S1130DD0B0FBF1F00AE0C3F3C551491CB0FBF1F0DC
S1130DE004E0C2F3C351491CB0FBF1F070BC70477E
S1130DF001001000020010000001100000021000A9
S1130E000004100000011010000210100004101063
S1130E1000401010005010200100002002000020AB
S1130E200400002008000020100000202000002002
S1130E30400000208000002000010020004000103D
S1130E40001010100001102080000030100000304D
S1130E50000100100002001010000010200000101B
S1130E6020000030010010100200101004001010C7
S1130E70080010100100001002000010040000100F
S1130E80010010200010100000E00F400000FF706F
S1130E900FC8FFFF8FDFFF7F30200080FCFF3FF88B
S1130EA00300C0070000404000080080C0E1E400E7
S1130EB00000011000000310001BB7000024F40020
S1130EC070383900C0C62D0000093D00433A5C5714
S1130ED06F726B5C736F6674776172655C4F70657B
S1130EE06E424C545C5461726765745C44656D6F0A
S1130EF05C41524D434D335F4C4D33535F454B5F23
S1130F004C4D3353383936325F4941525C426F6F2E
S1130F10745C6C69625C6472697665726C69625C4B
S1130F2073797363746C2E630000000000E10F405A
S1130F3004E10F4008E10F4040420F0000201C0074
S1130F4080841E0000802500999E360000403800F1
S1130F5000093D0000803E0000004B00404B4C0067
S1130F6000204E00808D5B0000C05D00008070009A
S1130F7000127A0000007D0080969800001BB700E4
S1130F800080BB00C0E8CE00647ADA000024F400DC
S1130F900000FA004FF0FF305C4908605C490860CB
S1130FA0704770B504460D46164600F045F9FF2813
S1130FB005D02819401E00F03FF9FF2801D1002078
S1130FC070BD600A4002B0F5804F2B463246214680
S1130FD003D14F48BDE870409CE04C48BDE87040E8
S1130FE098E070B504460D4600F026F90646281927
S1130FF0401E00F021F9FF2E01D0FF2801D100206E
S113100070BD01463046BDE87040E7E080B5404819
S1131010016811F1010F01D1012002BD416882680C
S11310205118C268511802695118426951188269ED
S11310305118C0694018C043401C00906A460421FE
S113104044F2F000FFF7ADFF02BD4FF480400168A9
S11310504268511882685118C268511802695118BF
S1131060426951188069401844F2F001096808186F
S1131070401E8041C00F704780B52548016811F1BA
S1131080010F03D000F084F8002808D01F4801683D
S113109011F1010F05D000F07BF8002801D10020E8
S11310A002BD012002BD4FF48040704780B5CA05DF
S11310B001D0002002BD02688A4201D1012002BD94
S11310C001604FF40072001D00F08CF9012002BD94
S11310D038B504460D460E48844208D10B4C2946C7
S11310E02046FFF7E3FF00280DD1002032BDB5F5FF
S11310F0804F01D10446F2E7204600F049F8002869
S1131100EDD1002032BD204632BD00004808002049
S11311104C0A00202DE9F0410746884614461D4636
S11311204FEA58267602386810F1010F05D131468E
S11311303846FFF7BBFF00281DD03868B04205D001
S113114031463846FFF7C4FF070014D03868A8EBCF
S11311500000384400F10408FFF71BFC381DA8EB1D
S11311600000B0F5007F0AD306F500713846FFF79A
S1131170AFFF070001D1002008E007F1040814F8CC
S1131180010B08F8010B6D1EE6D10120BDE8F081CA
S1131190F8B504460125206800F04EF8FF2801D177
S11311A00020F2BD002600E0761C802E14D22168B7
S11311B011EB860704EB860040680090FFF7E9FB1B
S11311C004223946684600F03BF9002803D1386808
S11311D000998842E8D000252846F2BDF8B50D46AE
S11311E00246914224D30146022921D329461429D7
S11311F01ED200F03CF80446284600F038F80646B3
S1131200284600F04DF88019401E001B401C850A3A
S1131210ADB2002600E0761CB6B23746AF4209DA1A
S1131220FFF7B7FB04EB872000F0EEF80028F2D0BC
S11312300020F2BD0120F2BD38B50446002501E0CE
S11312406D1CEDB2122D10D2FFF7A3FB0FF280003C
S113125005EB450100EB810001688C42F0D3426844
S113126051188C42ECD2007A32BDFF2032BD38B521
S11312700446002500E06D1CEDB2122D0DD2FFF7DF
S113128088FB05EB450080000FF244010A18127A2E
S113129023469A42EFD1085832BD4FF0FF3032BD99
S11312A038B50446002500E06D1CEDB2122D0DD2B8
S11312B0FFF76FFB0FF2180005EB450100EB81000F
S11312C0017A22469142EFD1406832BD002032BDFE
S11312D00040000000200000020000000060000048
S11312E00020000003000000008000000020000037
S11312F00400000000A00000002000000500000021
S113130000C00000002000000600000000E0000013
S11313100020000007000000000001000020000081
S11313200800000000200100002000000900000067
S113133000400100002000000A00000000600100DD
S1131340002000000B0000000080010000200000CD
S11313500C00000000A00100002000000D000000AF
S113136000C00100002000000E00000000E00100A9
S1131370002000000F0000000000020000800000B8
S11313801000000000800200008000001100000036
S11313900000030000800000120000000080030031
S11313A0008000001300000000F0D4B810B500F075
S11313B0DBF8002810D000F00DF900F052F900F02D
S11313C0D5F8064908400649086000F0CFF8001D2A
S11313D0046800F0C1F8A04710BD000080FFFF1FA3
S11313E008ED00E070B504460D46164605E015F814
S11313F0010B04F8010BFFF7CCFA3046461E80B20D
S11314000028F4D170BD000010B50446A00504D036
S113141084210FF2E000FFF703FADFF8C400012192
S113142041610460DFF8BC10816081688907FCD4E5
S1131430C068C00702D54FF0FF3010BD002010BDBA
S113144070B504460D46164615F0030F04D0C821A6
S11314500FF2A000FFF7E4F916F0030F04D0C9213E
S11314600FF29000FFF7DCF9DFF87400012141610D
S1131470DFF874100968C90727D5002E27D0E909B9
S1131480C9010160194B07E054F8041B05F07C0204
S11314909A1811602D1D361F15F07C0F02D1016BB7
S11314A0002901D1002EEFD111490162016AC90757
S11314B0FCD4E2E70560216841600D4981608168E0
S11314C0C907FCD4241D2D1D361F002EF2D1C0687F
S11314D0C00702D54FF0FF3070BD002070BD000082
S11314E000D00F40020042A4A0E10F4000D10F4001
S11314F0010042A4433A5C576F726B5C736F66746D
S1131500776172655C4F70656E424C545C546172D5
S11315106765745C44656D6F5C41524D434D335F48
S11315204C4D33535F454B5F4C4D33533839363252
S11315305F4941525C426F6F745C6C69625C6472B7
S1131540697665726C69625C666C6173686C696209
S11315502E63000072B6704762B67047FFF71ABD7B
S1131560FFF71FBDFFF73DBDFFF76FBDFFF79BBD45
S113157080B5FFF74BFD002801D1002002BDBDE876
S11315800140FFF779BD000010B500F081F800F0CC
S113159081FA2A4C0120207000F002FB0020207008
S11315A010BD10B5254C201D00F0C2FA012804D14D
S11315B001202070201D00F086F8201D00F029FB7A
S11315C0012806D100202070201DBDE8104000F045
S11315D07AB810BD704770B504460D46174E307882
S11315E0012803D1C9B2204600F07AFA30780028E5
S11315F004D12946C9B2204600F0E1FABDE87040A2
S113160000F05CB80D480078401E03D0401E01284D
S113161002D903E00820704700207047402070473B
S113162006480078401E03D0401E012802D903E07A
S113163008207047002070474020704700000020B9
S113164000F034B880B500F00CF80F484CF24F317C
S11316504160002181600521016000200B49086080
S113166001BD002008490860704707480068C003AE
S113167003D506480168491C0160704780B5FFF72F
S1131680F4FF0248006802BD10E000E0F00C002006
S1131690DFF884030021018000F1440100224A6044
S11316A080F843200A80114681707047DFF8680390
S11316B00178481E8041C043C00F70470020D649BE
S11316C081F84300704710B50178D34CFF2914D139
S11316D000F080F894F84300012802D1102000F0B3
S11316E070F8B4F94410012906DB012084F84300A2
S11316F0E01CBDE810404EE010BD2278012AFBD169
S1131700C92932D0CC293FD0CF293AD0D0292FD0E3
S1131710D12933D0D2292ED0F32917D0F4290FD0D0
S1131720F5290AD0F6290ED0FA2912D0FC2913D0B3
S1131730FD2914D0FE2915D029E000F0A3F8C9E74B
S113174000F0BDF8C6E700F094F8C3E700F0D6F85F
S1131750C0E700F07DF8BDE700F078F8BAE700F0E4
S113176065F8B7E700F056F8B4E700F0EDF8B1E734
S113177000F007F9AEE700F0D4F8ABE700F02EF97B
S1131780A8E700F03EF9A5E700F048F9A2E7202019
S113179000F017F89EE789B2FFF71DBF10B40023CD
S11317A003E00478E318DBB2401C0C46611E002CF5
S11317B0F7D11360012010BC70470020964948708F
S11317C070479549CA1CFE23137050700220A1F87B
S11317D04400704710B5FFF7F0FF8F4C01202070D4
S11317E0FF20E0701020207100206071FFF70AFFD5
S11317F0A071FFF715FFE071FFF712FF000A2072D6
S113180001206072A0720820A4F84400BDE81040D2
S1131810FFF7A4BE10B5804C00202070FFF7CDFF69
S1131820FF20E0700120A4F8440010BD7A48411C58
S1131830FF228A700022CA700A780A7100224A7153
S11318408A71CA710621A0F8441070470020B8E7D5
S11318507148C11CFF220A7044300FF2C412426066
S113186000224A708A70CA7007224A6008210180E7
S113187070476949FF22CA704431406848600120BA
S11318800880704770B50546FFF7BCFE6A78401EB5
S1131890904203DA2220BDE8704092E75E4E06F1E2
S11318A044046168301DFFF79DFDFF20F0706068FF
S11318B06978081860606878401C208070BD70B535
S11318C00446FFF79FFE401E6178884203DA222017
S11318D0BDE8704075E761684F4E06F144056960E4
S11318E06278301DFFF77EFDFF20F0706868617834
S11318F0081868606078401C288070BD38B5464977
S1131900CC1CFF22227001F14405CA1D416868689D
S1131910FFF744FF60700020A070E070082028806A
S113192031BD38B53C4CE51CFF20287000206870A0
S1131930A870FFF767FEE870002028716871A8712D
S11319400720A4F8440031BD70B50546FFF75AFEE0
S1131950314E06F144046A1C411E6068FFF700FE24
S1131960002803D13120BDE870402AE7FF20F07041
S1131970FFF748FE6168401E401860600120208027
S113198070BD38B50446FFF73DFE801E617888427D
S113199003DA2220BDE8324013E71F48FF21C1705B
S11319A000F14405012028806178080007D1FFF781
S11319B0DFFD002811D13120BDE8324001E7A21C2F
S11319C06868FFF7CDFD002803D13120BDE832401F
S11319D0F7E6686861780818686031BD38B50E4C60
S11319E004F1440541686868FFF7BCFD002803D191
S11319F03120BDE83240E4E6FF20E0700120288079
S1131A0031BD80B5FFF7D2FC0348FF21C17001212D
S1131A10A0F8441001BD00009C0C00203120D0E649
S1131A204F70656E424C540000B585B0042002909E
S1131A3010200090642302E00098401E009000985B
S1131A40002824D00820019001E0401E0190019854
S1131A500028F1D000994118491C009A521C5A439D
S1131A60B2FBF1F2D2B2413A0B2AEED21022B2FB0F
S1131A70F1F25143D1F11001E7D1042800D20290D0
S1131A80039269463548FEF71EFC012000E0002061
S1131A9005B000BD10B586B03148FFF72DF82F4CC6
S1131AA02046FEF7B0FBFFF7BFFF012804D08B21CF
S1131AB00FF2B000FEF7B4FE2046FEF7EFFB40F253
S1131AC06760009040F2FF7001900820029003903C
S1131AD002236A4601212046FEF7AEFC06B010BD83
S1131AE070B586B005460E461C4C01212046FEF713
S1131AF05DFC800704D5AE210FF26800FEF790FE6E
S1131B0040F2E17000900020029003960495034691
S1131B106A4602212046FEF78FFC01212046FEF78B
S1131B2045FC0546FEF735FFA807F6D406B070BDA0
S1131B3030B585B00446094D02212846FEF736FC2F
S1131B40C00701D4002007E0049401236A46194623
S1131B502846FEF756FD012005B030BD00000440C4
S1131B6000011000433A5C576F726B5C736F6674CC
S1131B70776172655C4F70656E424C545C5461725F
S1131B806765745C536F757263655C41524D434D78
S1131B90335F4C4D33535C63616E2E630000000071
S1131BA080B54848FEF7A8FFFFF753F860234FF4C9
S1131BB0614201464448BDE8005000F0B7B870B532
S1131BC004460D46412D04DB5B210FF20410FEF7A1
S1131BD027FE284600F062F8012804D05F210FF2A6
S1131BE0F000FEF71DFE00260DE0FEF7D2FEB6B2B1
S1131BF0A05D00F053F8012804D068210FF2D00052
S1131C00FEF70EFE761C3046294680B28842ECD39D
S1131C1070BD38B505462D4C607800280FD1201DC5
S1131C2000F02FF801282AD12079002827D0FFF7C7
S1131C3025FDA06400202070012060701FE0207842
S1131C402044401D00F01DF8012810D12078421CCA
S1131C50227010462179C0B2884210D1D2B2611DDF
S1131C602846FFF7BFFB00206070012032BDFFF75C
S1131C7005FDA16C6431814201D200206070002016
S1131C8032BD10B50446104800F00BF910F1010FF5
S1131C9002D02070012010BD002010BD10B50A4CE8
S1131CA00146204600F013F9002803D1002010BD9E
S1131CB0FEF76FFE204600F0DFF80028F8D0012080
S1131CC010BD00000100001000C00040500C0020B6
S1131CD0433A5C576F726B5C736F667477617265BD
S1131CE05C4F70656E424C545C5461726765745C01
S1131CF0536F757263655C41524D434D335F4C4D78
S1131D0033535C756172742E63000000DFF8EC11CC
S1131D10884207D0DFF8E811884203D0DFF8E411E5
S1131D20884201D10120704700207047F8B504466D
S1131D300E4617461D46FFF7E9FF002805D140F27D
S1131D400D110FF2D810FEF76BFD002F05D14FF4E3
S1131D5087710FF2C810FEF763FDDFF8AC0101686C
S1131D6011F0E04F19D0DFF8A41102680A40B2F173
S1131D70805F12D002680A40DFF894319A4203D19E
S1131D80026892B2022A08D002681140DFF8842166
S1131D90914204D10068000401D1102000E0082021
S1131DA07843864205D240F20F110FF27010FEF70D
S1131DB037FD204600F041F804F13000B6EB071F70
S1131DC0016804D241F0200101607F0802E021F0A3
S1131DD020010160F000B0FBF7F0401C40088109CD
S1131DE004F12402116000F03F0004F128010860AE
S1131DF004F12C000560002004F11801086020465D
S1131E00BDE8F240FFE710B50446FFF77FFF002866
S1131E1005D14FF4CF710FF20410FEF701FD04F168
S1131E202C00016841F01001016004F130000168E8
S1131E3040F201321143016010BD10B50446FFF7B2
S1131E4065FF002805D14FF4DF710FF2D000FEF7D3
S1131E50E7FC04F1180000680007FAD404F12C0030
S1131E60016821F01001016004F130000168DFF81D
S1131E70A8201140016010BD10B50446FFF746FFCD
S1131E80002805D140F2E9310FF29000FEF7C8FCBA
S1131E9004F118000068400900F0010080F001001E
S1131EA010BD10B50446FFF731FF002805D140F2FC
S1131EB009410FF26800FEF7B3FC04F11800006852
S1131EC0C00601D4206810BD4FF0FF3010BD38B5F6
S1131ED004460D46FFF71AFF002805D140F25B4186
S1131EE00FF23800FEF79CFC04F11800006880062D
S1131EF002D42560012032BD002032BD00C0004064
S1131F0000D0004000E0004000E00F400000FF70FF
S1131F100000011000000310FEFCFFFF433A5C5771
S1131F206F726B5C736F6674776172655C4F70651A
S1131F306E424C545C5461726765745C44656D6FA9
S1131F405C41524D434D335F4C4D33535F454B5FC2
S1131F504C4D3353383936325F4941525C426F6FCE
S1131F60745C6C69625C6472697665726C69625CEB
S1131F70756172746C69622E63000000B0F1402FC9
S1131F8043D0DFF8581288423FD0DFF85412884219
S1131F903BD0DFF85012884237D0DFF84C12884229
S1131FA033D0DFF8481288422FD0DFF84412884239
S1131FB02BD0DFF84012884227D0DFF83C12884249
S1131FC023D0DFF8381288421FD0DFF83412884259
S1131FD01BD0DFF83012884217D0DFF82C12884269
S1131FE013D0DFF8281288420FD0DFF82412884279
S1131FF00BD0DFF82012884207D0DFF81C12884289
S113200003D0DFF81812884201D101207047002064
S1132010704770B506460C461546FFF7AFFF00281B
S113202004D1E4210FF2F810FEF7FAFB002D08D0DA
S1132030012D06D0022D04D0E6210FF2E410FEF7A4
S1132040EFFB06F58060E907016801D5214300E054
S1132050A143016006F58460A907016801D5214305
S113206000E0A143016070BDF8B504460F46154673
S11320701E46FFF783FF002805D14FF4DD710FF2F0
S1132080A010FEF7CDFB012D0BD0022D09D0042D9D
S113209007D00C2D05D04FF4DF710FF28410FEF73A
S11320A0BFFB082E11D00A2E0FD00C2E0DD0092EF6
S11320B00BD00B2E09D00D2E07D0002E05D040F2E8
S11320C0C5110FF25C10FEF7ABFBF84304F5A061F9
S11320D0EA070A6801D53A4300E002400A6004F2C4
S11320E00451AA070A6801D53A4300E002400A6095
S11320F004F5A1616A070A6801D53A4300E0024089
S11321000A6004F5A3612A070A6801D53A4300E08E
S113211002400A6004F20C51F2070A6801D53A43FE
S113212000E002400A6004F5A261B2070A6801D522
S11321303A4300E002400A6004F2145172070A684C
S113214001D53A4300E002400A6004F21C51320710
S11321500A6801D53A4300E002400A6004F5A5612B
S1132160002E02D10868384301E00A681040086074
S1132170F1BD38B504460D46FFF700FF002805D130
S11321804FF464710FF29800FEF74AFB02222946CD
S11321902046FFF73EFF082304222946204601B0CB
S11321A0BDE8304060E738B504460D46FFF7E6FE6B
S11321B0002805D140F21F510FF26400FEF730FBF6
S11321C0022229462046FFF724FF0823012229463C
S11321D0204601B0BDE8304046E7000000800540DD
S11321E000500040009005400060004000A0054001
S11321F00070004000B005400040024000C00540AF
S11322000050024000D005400060024000E005405C
S11322100070024000F0054000D00340000006407A
S1132220433A5C576F726B5C736F66747761726567
S11322305C4F70656E424C545C5461726765745CAB
S113224044656D6F5C41524D434D335F4C4D335388
S11322505F454B5F4C4D3353383936325F494152F9
S11322605C426F6F745C6C69625C647269766572FF
S11322706C69625C6770696F2E6300003C210FF229
S11322800800FEF7CDBA0000433A5C576F726B5CEE
S1132290736F6674776172655C4F70656E424C54FF
S11322A05C5461726765745C44656D6F5C41524D4A
S11322B0434D335F4C4D33535F454B5F4C4D33536C
S11322C0383936325F4941525C426F6F745C7665CF
S11322D063746F72732E630080B500F005F800F02C
S11322E021F800F02EF8FCE780B50A48FEF722FC3E
S11322F00948FEF701FC03214FF04020FFF753FF8C
S11323000648FEF7F9FB03210548BDE80440FFF742
S113231030BF00008003C00101000020080000203D
S11323200070004080B5FFF73FF8FEF731FBFFF780
S113233089F9FFF713F9FFF727F9BDE8014000F029
S11323400BB880B5FEF725FBFFF78FF9FFF729F9E6
S1132350BDE8014000F009B810B50F4C0120207011
S1132360FFF78CF96060BDE8104010B5FFF768F91D
S1132370012810D0084C207801280CD1FFF77EF9F1
S1132380616801F5FA71884205D300202070BDE828
S11323901040FFF70BB810BDE80C002019E050F80E
S11323A0041BCB0744BFA9F101035918121F0023D2
S11323B0042A41F8043BF9D25FEA827C0B4604D537
S11323C04FF0000CA1F800C09B1CD10744BF0021B2
S11323D0197050F8042B002AE1D1704730B5016818
S11323E042688468014401EB5203D20748BF4C445D
S11323F0994201D10C3030BD11F9012B11F8015B68
S1132400002A04F8015B02D5521CF9D1F0E7521EF0
S1132410F4D5EDE710B5074979441831064C7C44EE
S1132420163404E00A68081D114488470146A14295
S1132430F8D110BD080000002400000061FFFFFF78
S1132440AC040000480800200000000091FFFFFFDA
S113245070000000080000000000002000F00BF8ED
S1132460002801D0FFF7D6FF0020AFF30080FFF76C
S113247033FF00F002F80120704700F001B80000BB
S11324800746384600F002F8FBE7000080B5AFF3DA
S11324900080024A11001820ABBEFBE726000200B0
S11324A0034B9D46AFF30080AFF30080FFF7D6FFE8
S11324B048080020AFF30080AFF30080FFF7CEFFA1
S10724C00004BD0053
S90324B523
